:020000040800F2
:10000000B01D002001010008E31C0008451B00088A
:10001000E11C000869010008391E0008000000000A
:10002000000000000000000000000000691D000842
:100030000105000800000000051D00086B1D0008F8
:100040001B0100081B0100081B0100081B01000820
:100050001B0100081B0100081B0100081B01000810
:100060001B0100081B0100081B0100081B01000800
:100070001B0100081B0100081B0100081B010008F0
:100080001B0100081B0100081B0100081B010008E0
:100090002D1E00081B0100081B0100081B010008A1
:1000A0001B0100081B0100081B0100081B010008C0
:1000B0001B0100081B0100081B0100081B010008B0
:1000C0001B0100081B0100081B0100081B010008A0
:1000D0001B0100081B0100081B0100081B01000890
:1000E0001B0100081B0100081B010008DFF80CD0F1
:1000F00000F028F800480047311F0008B01D00201C
:100100000648804706480047FEE7FEE7FEE7FEE7B1
:10011000FEE7FEE7FEE7FEE7FEE7FEE7E51D000877
:10012000ED000008202A04DB203A21FA02F0002129
:10013000704721FA02F3D040C2F1200291400843F7
:1001400019467047064C074D06E0E06840F0010391
:1001500094E8070098471034AC42F6D3FFF7CAFF83
:10016000B8260008D8260008FEE710B54FF4D8726C
:10017000036802EB01129B5813F00404436B9C606C
:100180000468436BA45856D0E4085C6003689A582E
:10019000436B02F00202DA604FF4DA72036802EB9A
:1001A00001129B58446B03F00F03236103689A58B4
:1001B000436BC2F30722DA614FF4DC72036802EB8F
:1001C00001129B58446B237503689B58446B1B0AB0
:1001D000637503689B58446B1B0CA37503689A589E
:1001E000436B120EDA754FF4DE72036802EB0112F4
:1001F0009B58446B237603689B58446B1B0A6376B9
:1002000003689B58446B1B0CA37603689A58436B96
:10021000120E0029DA76016810D00A6942F0200235
:100220000A6101684A6922F010024A6190F83910A7
:1002300022290CD010E0640D1C60A7E7CA6842F0C8
:100240002002CA6001684A6922F00202EDE70168F3
:100250004A6922F40F424A6190F83910322906D0D7
:10026000012180F8391000F075FC002010BD12212A
:10027000F7E700002DE9F14F86B0069800890828BD
:1002800053D9764E4FF0000B5946A6F802B00698A7
:1002900001F03EFE04460121069801F039FE552C7E
:1002A0007ED1AA287CD10221069801F031FE0446B5
:1002B0000321069801F02CFE05460521069801F061
:1002C00027FE07460421069801F022FE07EB0020D6
:1002D00080B20490162C28D10698018905F10900F6
:1002E0000590814221D3DFF878A155218AF80010CA
:1002F000AA218AF8011007218AF8021051218AF8F0
:100300000310411E069801F003FE564C4FF0010801
:10031000F0280DD00121069801F0D4FD86F8008068
:100320004CF20230A080F020A07007B0BDE8F08F42
:10033000291D069801F0ECFD0706691D069801F0DD
:10034000E7FD07EB0047A91D069801F0E1FD07EB6B
:100350000027E91D069801F0DBFD3844022705F16E
:100360000409009008E03946069801F0D1FD0AEB37
:1003700007017F1C8870BFB24F45F4D3A91D3848D0
:1003800000F076F8009981420FD086F800804CF298
:100390000230A080F120A070DDE9051007B000E078
:1003A0001AE0BDE8F04F01F08DBDDDE9051001F068
:1003B00089FD0498A0F20550B0F5005048D000F235
:1003C000FA304FF48065B0F5004008D0A0F5007019
:1003D0007A381ED07C2833D001210698DEE7A07839
:1003E0000128A2D084F8028086F800804CF20240F6
:1003F000A080DAF80F00E0601B4800F08BF81B4A81
:10040000002059461154401C80B2A842FAD3B18052
:100410008BE70220A07012480D30A0609AF80910F6
:100420009AF80A0001EB002080B2E080A84201D3D4
:10043000A4F806B04CF20220A08084F8008074E793
:100440000320A07086F800804CF20250A0806CE778
:100450000520A07086F8008067E7000014000020E7
:100460001C05002008010020003000081C010020AD
:1004700070B506464FF0FF300022094C0DE0B35C2A
:1004800058400023050E5B1C54F825509BB285EAAA
:100490000020042BF6D3521C92B28A42EFD370BDD7
:1004A000B8220008F0B58BB0002401254EF22000E0
:1004B0000594CDE906454EF2E0164FF6FF778DE83C
:1004C000D10069460D480895049400F0F9F808B188
:1004D00000F018F8CDE905544FF4604007958DE819
:1004E000D100694605480895049400F0E9F8002811
:1004F00001D000F007F80BB0F0BD0000C8000020EC
:10050000704700005FF0010484F3138800F016FFC9
:10051000FAE7000030B585B000250446049500F0E8
:10052000EBFC0D48844212D2401C001B800A039051
:1005300001210095CDE9011404A9684600F03EFCB4
:10054000044600F08FFC24B1012005B030BD00F05E
:1005500089FC0020F9E70000FFDF010810B500F07A
:10056000CBFC03493420C860BDE8104000F07ABCE1
:10057000002002402DE9F041164688460546002439
:1005800000F0BAFC0E4F13E058F82420002329464F
:10059000022000F071FC10B10320BDE8F08158F892
:1005A00024002968814201D00220F6E7641C2D1D39
:1005B000B44201D2BD42E7D900F054FC0020ECE780
:1005C000FBDF010806490020C8610648016941F0C7
:1005D00004010161016941F04001016170470000BF
:1005E0006800002000200240064A0021D16106492F
:1005F0000A6942F002020A614861086940F040005D
:10060000086170476800002000200240044B00226F
:10061000DA61044A136943F00103136101807047F2
:1006200068000020002002400E49C868C2060E483B
:1006300003D5C26942F00202C261CA68520703D5FB
:10064000C26942F00102C261CA69D20707D0C26919
:1006500042F00402C261C86920F00100C8611420A0
:10066000C8607047002002406800002070B5054651
:1006700000F0AAFD0646114C09E0681C07D025B120
:1006800000F0A2FD801BA84201D9032070BDE068E4
:10069000C007F2D1E068800601D52020E060E06864
:1006A000C00605D4E069C00702D1E068400703D561
:1006B000FFF7BAFF012070BD002070BD002002408E
:1006C000F0B50C7D012303FA04F20468D4F800525B
:1006D0004E6A25F47C5503EB06231D43C4F80052F3
:1006E0000368D3F81C429443C3F81C424FF41073C0
:1006F000CD691C1DBDB90568D5F80C629643C5F8D7
:100700000C628E894D684F6966F31F45066803EBDE
:10071000C707F5510E890D684F6966F31F450668D6
:1007200004EBC707F551CD69012D17D10568D5F840
:100730000C621643C5F80C620E884D684F6966F36B
:100740001F45066803EBC703F5500D89CB684E695A
:1007500065F31F43056804EBC6042B518B69002B1E
:100760000368D3F8044211D054EA0204C3F80442E7
:100770000B69002B0368D3F8144209D054EA020431
:10078000C3F81442096A012904D009E09443EDE753
:100790009443F5E70168D1F81C321343C1F81C32C9
:1007A0000068D0F8001221F00101C0F8001200200A
:1007B000F0BD10B504000BD0022084F839002046AB
:1007C00000F060F9002084F8390084F8380010BD8A
:1007D000012010BD0068416941F00201416170478C
:1007E00070B50168044648694FF00105C043C00771
:1007F00022D18A685B48904307D08A685A48904360
:1008000003D08A685948904316D14A69204622F09D
:1008100001024A6194F83910122904D101684A6929
:1008200022F40F424A6190F83910322922D080F820
:10083000395000BF00F090FA20684169C943890728
:1008400006D4C068800703D000212046FFF78DFC46
:1008500020684169C943C90606D40069800703D0EE
:1008600001212046FFF781FC20688169C943C9073F
:1008700004D00FE0222180F83910DBE74169C94339
:10088000C90507D44169C943090403D4E16B41F0A8
:100890000101E1638169C94389070BD44169C943F7
:1008A000890507D44169C943090403D4E16B41F0C8
:1008B0000201E1638169C94349070BD44169C94316
:1008C000490507D44169C943090403D4E16B41F0E8
:1008D0000401E163816911F0700F25D04169C943BA
:1008E000090521D44169C94309041DD4816901F076
:1008F000700140292AD006DC102909D020290BD00C
:1009000030290DD11EE0502924D0602908D125E0DE
:10091000E16B41F0080102E0E16B41F01001E1639D
:10092000816921F070018161E06B002809D02068A5
:10093000416841F00401416084F839502046FFF7D6
:1009400049FF70BDE16B41F02001E8E7E16B41F048
:100950004001E4E7E16B41F08001E0E7E16B41F445
:100960008071DCE7030000040003000800000310AE
:100970002DE9F04104004FF0000504D094F839004F
:10098000002618B107E00120BDE8F08184F8386046
:10099000204600F093F8022084F8390020680168AE
:1009A00021F0020101602068016841F0010101604D
:1009B00000F00AFC07464FF0030804E000F004FCD6
:1009C000C01B0A2845D820684068C007F6D02068B8
:1009D0004168C9074BD0A169012901D145F08005C3
:1009E000E169012901D145F04005216A012901D1C0
:1009F00045F02005616A012901D145F01005A16A81
:100A0000012901D145F00805E16A012901D145F02C
:100A10000405016821F0FC0129430160D4E90201C9
:100A20000843D4E90412114308436168491E08438E
:100A30002168C8612068016821F00101016000F0AF
:100A4000C3FB05460BE000BF00F0BEFB401B0A28BD
:100A500005D984F8398084F83860032094E7206849
:100A60004068C007F0D120684068C00703D0042068
:100A700084F8390087E7E663012084F83900002014
:100A800082E7000010B50068094988420ED1094884
:100A9000C16921F00071C1614FF44071064800F056
:100AA0003DFABDE81040142000F000BC10BD00006D
:100AB0000064004000100240000C014010B50068C6
:100AC0001F4986B0884239D11E48C16941F0007182
:100AD000C161C0691C4C00F0007004904FF480703C
:100AE00000900020019002906946204600F088FAAC
:100AF0006015009002200190032003906946204673
:100B000000F07EFA1148416821F4C04141F480416F
:100B1000416000221146142000F0DEFB142000F09A
:100B2000D0FB0B4800F1400420631C306063FFF7EA
:100B3000B9FC2068416941F00201416106B010BD75
:100B40000064004000100240000C01400000014021
:100B500088000020F0B5406B194A816849BB0169E3
:100B600039B30068A0F5E063513B22D1CCB200213B
:100B700014480D4601261AE0576B01F11403B0F832
:100B800004C0FB5CC76807F80C3083885B1C9FB20D
:100B9000878043889F4200D3858007897F1CBFB22E
:100BA00007819F4201D903818672491CC9B2A142C3
:100BB000E2D31068416941F002014161F0BD0000DB
:100BC000C8000020540000202DE9F05F044690F892
:100BD00038000E46012813D04FF0010884F8388001
:100BE00094F8390022280ED05FF0120084F8390002
:100BF000216888684FF00007400106D500250DE008
:100C00000220BDE8F09F3220F0E78868000101D59E
:100C1000012503E08868C00055D502254FF4C07057
:100C200000EB05100A5802F001020A50216B8A6895
:100C3000EAB3D4F800C05CF800301343CA684968CE
:100C400042EAC1010B434CF80030216B0A7C02F0F0
:100C50000F020A614FF4C271226801EB051153586B
:100C600023F00F03535022685358D4F830C0DCF8F7
:100C700010C043EA0C035350216B4FF4C47303EBD1
:100C800005130A7DD1F8151042EA01222168CA50E5
:100C9000216B4FF4C67303EB05130A7ED1F81910CC
:100CA00042EA01222168CA5021680A5800E011E096
:100CB00042F001020A5000F087FA8146DFF88CA06A
:100CC000DFF88CB020E0042084F8390084F8387014
:100CD000012096E722681358D1F80CC0098843EA2E
:100CE0000C0343EA41511150AFE7701C0CD02EB1F8
:100CF00000F06AFAA0EB0900B04205D9032084F89D
:100D0000390084F838707CE795B12068012D81683E
:100D100013D0104888430028E7D194F839003228CE
:100D20000ED084F8398000BF84F83870002068E75E
:100D3000206881682AEA0100EDE72BEA0100EAE772
:100D4000222084F8390084F83870EDE703000004AD
:100D50000003000800000310704710B5040002D023
:100D6000607910B106E0012010BD002020712046FE
:100D700000F004F801206071002010BD08B5006883
:100D80000649884208D10648416941F04001416165
:100D9000406900F04000009008BD000000300240B3
:100DA0000010024031B500F00FFA044600F00CFAD2
:100DB0000099001B8842F9D338BD00002DE9F047A7
:100DC000054626480F460126017E01290FD0012144
:100DD000814601762868DFF888804CF2503402287A
:100DE00008D0A2462046FFF741FCA8B131E002201E
:100DF000BDE8F0872046FFF739FC08BB0120FFF76C
:100E0000E1FB2046FFF732FCD8F81010064621F02F
:100E10000401C8F810101CE04FF0FF303860AC68D7
:100E200011E02046FFF7E0FB5046FFF71FFCD8F823
:100E30001010060021F00201C8F8101001D03C602B
:100E400007E004F58064D5E9020100EB8120A042AF
:100E5000E7D8002189F818103046C9E7680000205B
:100E6000002002400348016941F080010161002037
:100E700070470000002002402DE9F05F07461C4843
:100E800088460024017E15461E46012909D001210D
:100E9000814601764CF2503A5046FFF7E7FB18B115
:100EA00022E00220BDE8F09F012F02D0022F00D0E7
:100EB0000427D346DFF83CA0220128463146FFF73D
:100EC00031F981B208EB4400FFF7A0FB5846FFF769
:100ED000CDFBDAF8102022F00102CAF8102018B970
:100EE000641CE4B2BC42E7D3002289F81820D9E799
:100EF000680000200020024005480169090605D568
:100F00000449416004494160002070470120704756
:100F10000020024023016745AB89EFCD2DE9F04366
:100F200000230F24DFF8C0C059E001229A400A4094
:100F300054D0FF2A01D8074601E000F104074FEA28
:100F4000830601D9A6F12006D7F8008004FA06F539
:100F50004FF0040928EA050809FA06F948EA0908E1
:100F6000C7F80080C56825EA0205C56023F00305BF
:100F70006544AF684FEA83764FEA167604FA06F9BD
:100F800009EA0708194FB84201D100270FE0184FAE
:100F9000B84201D101270AE0164FB84201D1022719
:100FA00005E0154FB84201D1032700E00427B74000
:100FB000474513D1AF6827EA0907AF600F4D2E6888
:100FC00096432E602D1D2E6896432E602D1D2E6893
:100FD00096432E602D1D2E6896432E605B1C31FAC1
:100FE00003F2A2D1BDE8F0830000014000080140F7
:100FF000000C0140001001400014014000040140B9
:101000002DE9F84FDFF890A100220AF1040B1446F5
:1010100001274FF00F090BF1040E00BF0B6807FA10
:1010200004F52B40AB4274D1DFF870C14E68A6EBDB
:101030000C0866452BD00DDC032E34D005DC36B30E
:10104000012E19D0022E2FD11BE0112E16D0122EF8
:101050002AD119E0B8F5881F19D006DCB8F5803F11
:1010600015D0B8F5801F1FD111E0B8F5001F0ED0C4
:10107000B8F5041F18D10AE0CA6815E0CA68121D45
:1010800012E0CA6808320FE0CA680C320CE08A68C5
:101090002AB1012A4FF0080203D0456104E004227E
:1010A00002E0056100E00022FF2B01D8064601E0C6
:1010B00000F104064FEA840501D9A5F12005D6F810
:1010C00000C009FA05F82CEA080C02FA05F54CEA0A
:1010D000050CC6F800C04D68ED0057D5304DAE691F
:1010E00046F00106AE61AD6924F0030605F0010586
:1010F00000952C4D06EB050CDCF80850A6074FEACE
:10110000167809FA08F6B543274EB04202D10026F8
:1011100010E03BE0254EB04201D101260AE0244E0A
:10112000B04201D1022605E0224EB04201D1032691
:1011300000E0042606FA08F62E43CCF808604D6855
:10114000DAF80060ED03554601D51E4300E09E43EA
:101150002E604D68DBF80060AD035D4601D51E438F
:1011600000E09E432E604D68DEF80060ED0275469B
:1011700001D51E4300E09E432E604D68AD020E4D2A
:101180002E6801D51E4300E09E432E60641C102C87
:10119000FFF444AFBDE8F88F0004014000001110D7
:1011A000001002400000014000080140000C014016
:1011B00000100140001401400C0401400AB101611B
:1011C00070470904FBE70000014800687047000011
:1011D0000000002002480168491C016070470000BF
:1011E00000000020074810B5016841F010010160BF
:1011F000032000F091F8002000F006F800F016F847
:10120000002010BD0020024010B5044600F06CF92B
:101210004FF47A71B0FBF1F000F07CFC0022214623
:10122000501E00F059F8002010BD00001D4808B500
:10123000816941F001018161806900F00100009045
:10124000032000F069F8002211466FF00B0000F057
:1012500043F8002211466FF00A0000F03DF800222A
:1012600011466FF0090000F037F800221146501FB8
:1012700000F032F800221146101F00F02DF8002275
:101280001146901E00F028F800221146501E00F072
:1012900023F80548416821F0E06141F000714160A8
:1012A00008BD0000001002400000014000F01F02D5
:1012B000012191404009800000F1E020C0F8801138
:1012C000704700F01F02012191404009800000F1A9
:1012D000E020C0F800117047F0B40E4B1B680C46BC
:1012E000C3F30223C3F10705042D00D90425191DFA
:1012F000072901D2002300E0DB1E012606FA05F1D2
:10130000491E214099409E40761E16403143F0BC54
:1013100000F0E8BC0CED00E0064900F007020868A8
:101320004FF6FF03184040EA0220034A10430860CA
:10133000704700000CED00E00000FA05BFF34F8F8E
:1013400005480168054A01F4E06111430160BFF3FB
:101350004F8F00BFFDE700000CED00E00400FA0530
:101360002DE9F047DFF8708105460E46D8F80000F9
:1013700000F00700B0420CD2D8F8001021F00701AD
:101380003143C8F80010D8F8000000F00700B04260
:1013900077D12878514C800705D56068A96820F07E
:1013A000F000084360602878C00759D069680120C0
:1013B00001290DD0022929D05FF0020393FAA3F28C
:1013C000B2FA82F242F02002520904D0226803E00D
:1013D0004FF40033F2E7626A93FAA3F3B3FA83F3AC
:1013E00003F01F03984002424BD0606820F00300D6
:1013F00008436060FFF7E8FE6968074641F28830FD
:1014000001290DD00229814617D025E04FF0007345
:10141000D4E700BFFFF7D8FEC11B494501D918E04A
:1014200081466068C0F381000128F3D118E000BF55
:10143000FFF7CAFEC11B49450BD86068C0F38100A5
:101440000228F5D10CE000BFFFF7BEFEC11B4945E5
:1014500002D90320BDE8F087606810F00C0FF3D1CB
:10146000D8F80010404601F00701B1420BD90168DD
:1014700021F0070131430160006800F00700B0422D
:1014800001D00120E6E72878400705D56068E968C3
:1014900020F4E060084360602878000706D56068A3
:1014A000296920F4605040EAC100606000F022F831
:1014B0006168F02292FAA2F201F0F001B2FA82F22F
:1014C000D140074A515CC840064908600020FFF738
:1014D0009BFE0020BEE700000020024000100240FA
:1014E000A82200080C000020014800687047000096
:1014F0000C00002010B519A385B00FCB8DE80F00AC
:101500001AA01B4B006804905A681A4802F00C019C
:1015100004291DD008291BD14FF4701494FAA4F4A7
:1015200002F47011B4FA84F4E140D2031DF8011002
:1015300010D55A684FF4003393FAA3F302F4003243
:10154000B3FA83F3DA4004AB9A5CB0FBF2F04843A1
:1015500005B010BD08484843FAE70000020304053F
:10156000060708090A0B0C0D0E0F101001020000EF
:101570000010024000127A0000093D002DE9F84FEA
:1015800004460078F74DC0074FF0010625D0686883
:101590007704C0F38100012807D06868C0F3810098
:1015A00002281BD16868C00318D597FAA7F0B0FAD3
:1015B00080F040F02000400901D0286800E0686A0F
:1015C00097FAA7F1B1FA81F101F01F0106FA01F1D2
:1015D00008425ED0606800287CD05AE06068B0F5B0
:1015E000803F0BD010B1B0F5A02F11D0286820F4A7
:1015F00080302860286820F4802002E0286840F4C9
:1016000080302860606828B3FFF7DEFD80460BE07D
:10161000286840F480202860F0E700BFFFF7D4FD81
:10162000A0EB0800642871D897FAA7F0B0FA80F010
:1016300040F02000400901D0286800E0686A97FA6D
:10164000A7F1B1FA81F101F01F0106FA01F1084298
:10165000E4D01EE0FFF7B8FD804605E0FFF7B4FDDB
:10166000A0EB08006428DED897FAA7F0B0FA80F063
:1016700040F02000400901D0286800E0686A97FA2D
:10168000A7F1B1FA81F101F01F0106FA01F1084258
:10169000E4D12078DFF8D08280074FF000094FF0C6
:1016A00002075BD568684FF0F80B10F00C0F07D0FD
:1016B0006868C0F3810002281CD16868C00319D48F
:1016C00097FAA7F0B0FA80F040F02000400902D06D
:1016D000286801E08BE0686A97FAA7F1B1FA81F116
:1016E00001F01F0106FA01F108422CD020690128FF
:1016F0007DD128E0206990B396FAA6F0B0FA80F088
:1017000048F82060FFF760FD824607E011E100BF66
:10171000FFF75AFDA0EB0A00022884D897FAA7F039
:10172000B0FA80F040F02000400901D0286800E0C5
:10173000686A97FAA7F1B1FA81F101F01F0106FA80
:1017400001F10842E4D028689BFAABF26169B2FA71
:1017500082F220F0F80091400843286025E0FFE77E
:1017600096FAA6F1B1FA81F148F82190FFF72CFD25
:10177000824605E0FFF728FDA0EB0A000228CCD83E
:1017800097FAA7F0B0FA80F040F02000400901D0AD
:10179000286800E0686A97FAA7F1B1FA81F101F0D0
:1017A0001F0106FA01F10842E4D1207800076ED546
:1017B000A069B8B396FAA6F0B0FA80F008EB800002
:1017C000C0F88064FFF700FD824605E0FFF7FCFCEF
:1017D000A0EB0A000228A0D897FAA7F0B0FA80F090
:1017E00040F06000B6EB501F02D128680CE062E1C7
:1017F00097FAA7F0B0FA80F040F06000B7EB501F06
:1018000001D1286A00E0686A97FAA7F1B1FA81F17C
:1018100001F01F0106FA01F21042D7D00120FFF7B4
:10182000C1FA34E0FFE796FAA6F1B1FA81F108EBCC
:101830008101C1F88094FFF7C7FC824606E000BF33
:10184000FFF7C2FCA0EB0A00022872D897FAA7F0B3
:10185000B0FA80F040F06000B6EB501F01D128686C
:101860000BE097FAA7F0B0FA80F040F06000B7EB19
:10187000501F01D1286A00E0686A97FAA7F1B1FA0F
:1018800081F101F01F0106FA01F21042D8D120784F
:10189000400765D5E86940F08050E861E869DFF805
:1018A000CCB000F080500090DBF8001041F4807163
:1018B000CBF80010FFF788FC824605E0FFF784FCB8
:1018C000A0EB0A00642834D8DBF80000C005F5D589
:1018D000E06801280AD008B1052813D0286A20F052
:1018E00001002862286A20F0040002E0286A40F023
:1018F00001002862E06841F2883B90B3FFF764FC86
:1019000082460BE0286A40F004002862EEE700BF40
:10191000FFF75AFCA0EB0A0159450AD897FAA7F03D
:10192000B0FA80F040F04000B6EB501F02D12868BA
:101930000CE0A3E097FAA7F0B0FA80F040F0400086
:10194000B7EB501F01D1286A00E0686A97FAA7F147
:10195000B1FA81F101F01F0206FA02F10842D7D074
:1019600031E005E0001002400000424200700040FB
:10197000FFF72AFC824605E0FFF726FCA0EB0A01F0
:1019800059457BD897FAA7F0B0FA80F040F04000B4
:10199000B6EB501F01D128680BE097FAA7F0B0FA18
:1019A00080F040F04000B7EB501F01D1286A00E002
:1019B000686A97FAA7F1B1FA81F101F01F0206FAFD
:1019C00002F10842D8D1E06980B36968C1F38101AE
:1019D000022970D04FF080714F000228484609D08C
:1019E00091FAA1F1B1FA81F148F82100FFF7ECFB7F
:1019F000044669E08A4691FAA1F1B1FA81F1C14643
:101A000048F82100FFF7E0FB804605E0FFF7DCFB2C
:101A1000A0EB0800022854D897FAA7F0B0FA80F09B
:101A200040F02000400902D0286801E061E0686AC7
:101A300097FAA7F1B1FA81F101F01F0106FA01F15D
:101A40000842E3D1206AB0F5803F05D16868A168FB
:101A500020F4003008436860D4E90801084369684D
:101A600021F47411084368609AFAAAF0B0FA80F081
:101A700049F82060FFF7A8FB044606E021E000BF1C
:101A8000FFF7A2FB001B02281BD897FAA7F0B0FAB9
:101A900080F040F02000400901D0286800E0686A2A
:101AA00097FAA7F1B1FA81F101F01F0106FA01F1ED
:101AB0000842E5D01DE01EE0FFF786FB001B022870
:101AC00002D90320BDE8F88F97FAA7F0B0FA80F0AA
:101AD00040F02000400901D0286800E0686A97FAC9
:101AE000A7F1B1FA81F101F01F0106FA01F10842F4
:101AF000E2D10020E6E70120E4E74FF0E0210428EE
:101B0000086903D020F004000861704740F0040029
:101B1000FAE7704710B5401EB0F1807F01D3012075
:101B200010BD4FF0E02460610F21601700F0DAF87B
:101B30000020A06107202061002010BD10B5FFF734
:101B4000E8FF10BD5FF0010484F31388FFF7F6FB94
:101B5000FAE7000002494AF6AA2008607047000030
:101B60000030004001B481B0019800680949084084
:101B7000B0F1005F03D0012002B0FFF713B9019864
:101B800040680549009008600199096881F3088858
:101B900002B000470000FE2F100000200F4810B5D3
:101BA0000D4901603021416000214FF440328160D5
:101BB000C0E9031201224161C0E90612C0E908210F
:101BC0008162C162FEF7D4FE002803D0BDE8104058
:101BD000FEF798BC10BD000000640040C800002063
:101BE000074910B5054808600846FFF7B6F8002811
:101BF00003D0BDE81040FEF785BC10BD00300240A8
:101C000004000020F0B5294885B0816941F0100139
:101C10008161816901F010010491816941F0040141
:101C20008161816901F004010491816941F0080139
:101C3000816180691E4D00F008000490002240215F
:101C40002846FFF7BBFA1B4E002210213046FFF753
:101C5000B5FA4FF460400324CDE900046946164804
:101C6000FFF7CEF949F6BF70CDE900046946284672
:101C7000FFF7C6F94FF6EF40CDE90004694630465C
:101C8000FFF7BEF940200124CDE900040227694690
:101C900003972846FFF7B4F91020CDE90004694600
:101CA00003973046FFF7ACF905B0F0BD00100240D5
:101CB00000080140000C014000100140074845F2B7
:101CC000555101600421416040F6C41181604AF61B
:101CD000AA2101604CF6CC41016070470030004001
:101CE000FEE770470907090E002806DA00F00F002A
:101CF00000F1E02080F8141D704700F1E02080F82A
:101D0000001470477047000003488188491C818097
:101D10004188491C418070471400002030B50E48AE
:101D20000068816841F0010181600C480C4A0D4B4C
:101D3000C168091F8C08002004E000BF52F8205041
:101D40001D60401CA042F9D318688958814201D017
:101D5000002030BD012030BD04000020080100201B
:101D60000030000800300240704710B5FFF7CCFF8C
:101D7000FFF730FABDE81040FFF7E0BE30B58FB096
:101D800001210804CDE900100024029402250491E9
:101D9000CDE907504FF4E01009906846FFF7EEFBDD
:101DA00058B90F20CDE90A056802CDE90C4002219F
:101DB0000AA80E94FFF7D4FA08B1FEF7A3FBFFF7C9
:101DC00093FB4FF47A71B0FBF1F0FFF7A3FE042010
:101DD000FFF793FE00221146501EFFF77DFA0FB069
:101DE00030BD00000D48016841F00101016041680B
:101DF0000B4A1140416001680A4A114001600168C4
:101E000021F480210160416821F4FE0141604FF41A
:101E10001F0181600449C003086070470010024040
:101E20000000FFF8FFFFF6FE08ED00E00148FEF7B6
:101E3000D7BC0000C8000020FEE700000B4D0C4C92
:101E4000FFF788FE0B48FEF715FA00F08FF900F057
:101E5000BDF900F0A3F968780128F1D10648FEF732
:101E6000A8FC2046FFF77EFEEAE7000008010020FC
:101E70000030000854000020C800002010B5FEF714
:101E80006DFB064900204FF47A728870C880087094
:101E90004870087402498A80488010BD08010020FB
:101EA0001400002002E008C8121F08C1002AFAD15D
:101EB00070477047002001E001C1121F002AFBD1CA
:101EC0007047000010B5114B04891A688C4208D382
:101ED000546924F0020454610289521A07E0C18057
:101EE00010BD516921F00201516101890022028176
:101EF0001A68536943F002035361C288114442884F
:101F000089B28A42EBD8891A89B2E8E7C800002072
:101F100002898A4208D3C2881144428889B28A421F
:101F200003D8891A89B200E00021C068405C70477C
:101F3000FFF758F9FFF722FFFFF764FEFFF72EFEC9
:101F4000FFF74EFEFFF7BAFEFFF798FFFFF776FFA9
:101F5000FEE7000070B50B212448FEF789FA234CF8
:101F6000010E244DE172010C2173010A6173A0730B
:101F70001F48296B00880860296B0020C860296B06
:101F80008860296B08200861296B20780875296B07
:101F900060784875022021182B6B8A7800F11401B3
:101FA000401CC0B25A540828F5D314211148FEF73A
:101FB0000BFE012801D1FFF7F1FD296B0620086116
:101FC000002021182B6B8A7A00F11401401CC0B24A
:101FD0005A540628F5D314210648FEF7F5FD0128CA
:101FE00003D1BDE87040FFF7D9BD70BD32000020BD
:101FF00054000020C800002070B511212C48FEF7C5
:1020000037FA2B4D010E2C4C6974010CA974010A8E
:10201000E97428752748216B082600880860206B22
:102020000661216B28780875216B68784875022055
:102030002918236B8A7800F11401401CC0B25A544D
:102040000828F5D314211C48FEF7BEFD012801D154
:10205000FFF7A4FD206B066100202918236B8A7A04
:1020600000F11401401CC0B25A540828F5D31421C1
:102070001148FEF7A9FD012801D1FFF78FFD216B63
:102080000420086100202918236B8A7C00F11401C8
:10209000401CC0B25A540428F5D314210648FEF758
:1020A00093FD012803D1BDE87040FFF777BD70BDF7
:1020B0001C00002054000020C800002070B5284CEF
:1020C000020AA271E0712172080A60720A21204698
:1020D000FEF7CEF9010EA172010CE172010A214D49
:1020E00021736073296B0020C860296B88601E48CB
:1020F000296B00880860296B08200861296B20780B
:102100000875296B60784875022021182B6B8A7836
:1021100000F11401401CC0B25A540828F5D3142110
:102120001048FEF751FD012801D1FFF737FD296B5B
:1021300005200861002021182B6B8A7A00F1140118
:10214000401CC0B25A540528F5D314210548FEF7A7
:102150003BFD012803D1BDE87040FFF71FBD70BDF6
:1021600042000020C8000020540000200948817867
:1021700000290ED1017C042909D2074A9388322B09
:1021800007D300239380491C0174FFF735BF012159
:102190004170704708010020140000200948417870
:1021A00000290ED1817800290BD007494A88B2F561
:1021B0007A7F06D900224A80C1884CF20230FFF7AC
:1021C0007DBF704708010020140000202DE9F04772
:1021D000324E012700253078314C012825D1357049
:1021E0002046A1788088012906D0022906D003293B
:1021F00008D0052919D113E0002100E0E188FFF79C
:102200005DFF12E0FFF78AFD012803D000214CF2A8
:102210000230F4E7A0880021FFF750FF677004E068
:10222000FFF798FEA570657025742078012831D1DC
:102230002570E188A846481E4CF20269B0F5806F0F
:102240002AD2174D1335485D48B14CF20220FFF7F2
:1022500035FFE1214846BDE8F047FFF72FBF1148A1
:10226000A36800EBC11020221946FEF783F960B184
:102270004C464FF47A75EE212046FFF71FFFFFF71B
:1022800069FC2846FEF78EFDF5E7E0884755377074
:10229000A6F80280BDE8F087E221DBE71400002009
:1022A00008010020802F000800000000000000004E
:1022B000010203040607080900000000B71DC1045D
:1022C0006E3B8209D926430DDC7604136B6BC51770
:1022D000B24D861A0550471EB8ED08260FF0C922E8
:1022E000D6D68A2F61CB4B2B649B0C35D386CD3150
:1022F0000AA08E3CBDBD4F3870DB114CC7C6D0481C
:102300001EE09345A9FD5241ACAD155F1BB0D45BF7
:10231000C2969756758B5652C836196A7F2BD86E5F
:10232000A60D9B6311105A6714401D79A35DDC7DD7
:102330007A7B9F70CD665E74E0B6239857ABE29CC3
:102340008E8DA191399060953CC0278B8BDDE68FF7
:1023500052FBA582E5E66486585B2BBEEF46EABADF
:102360003660A9B7817D68B3842D2FAD3330EEA9D7
:10237000EA16ADA45D0B6CA0906D32D42770F3D03B
:10238000FE56B0DD494B71D94C1B36C7FB06F7C36F
:102390002220B4CE953D75CA28803AF29F9DFBF667
:1023A00046BBB8FBF1A679FFF4F63EE143EBFFE54F
:1023B0009ACDBCE82DD07DEC77708634C06D473067
:1023C000194B043DAE56C539AB0682271C1B43236F
:1023D000C53D002E7220C12ACF9D8E1278804F16E7
:1023E000A1A60C1B16BBCD1F13EB8A01A4F64B054F
:1023F0007DD00808CACDC90C07AB9778B0B6567C1B
:1024000069901571DE8DD475DBDD936B6CC0526FF6
:10241000B5E6116202FBD066BF469F5E085B5E5A5E
:10242000D17D1D576660DC5363309B4DD42D5A49D6
:102430000D0B1944BA16D84097C6A5AC20DB64A88A
:10244000F9FD27A54EE0E6A14BB0A1BFFCAD60BBF6
:10245000258B23B69296E2B22F2BAD8A98366C8EDE
:1024600041102F83F60DEE87F35DA9994440689DD6
:102470009D662B902A7BEA94E71DB4E0500075E43A
:10248000892636E93E3BF7ED3B6BB0F38C7671F76E
:10249000555032FAE24DF3FE5FF0BCC6E8ED7DC266
:1024A00031CB3ECF86D6FFCB8386B8D5349B79D14E
:1024B000EDBD3ADC5AA0FBD8EEE00C6959FDCD6DBC
:1024C00080DB8E6037C64F643296087A858BC97E72
:1024D0005CAD8A73EBB04B77560D044FE110C54BE2
:1024E000383686468F2B47428A7B005C3D66C15852
:1024F000E4408255535D43519E3B1D252926DC2136
:10250000F0009F2C471D5E28424D1936F550D832F9
:102510002C769B3F9B6B5A3B26D6150391CBD40759
:1025200048ED970AFFF0560EFAA011104DBDD014D9
:10253000949B93192386521D0E562FF1B94BEEF53D
:10254000606DADF8D7706CFCD2202BE2653DEAE6F9
:10255000BC1BA9EB0B0668EFB6BB27D701A6E6D3D9
:10256000D880A5DE6F9D64DA6ACD23C4DDD0E2C0D9
:1025700004F6A1CDB3EB60C97E8D3EBDC990FFB915
:1025800010B6BCB4A7AB7DB0A2FB3AAE15E6FBAA71
:10259000CCC0B8A77BDD79A3C660369B717DF79F61
:1025A000A85BB4921F4675961A163288AD0BF38C51
:1025B000742DB081C330718599908A5D2E8D4B59F1
:1025C000F7AB085440B6C95045E68E4EF2FB4F4A71
:1025D0002BDD0C479CC0CD43217D827B9660437FE1
:1025E0004F460072F85BC176FD0B86684A16476C51
:1025F00093300461242DC565E94B9B115E565A1535
:1026000087701918306DD81C353D9F0282205E06F8
:102610005B061D0BEC1BDC0F51A69337E6BB523358
:102620003F9D113E8880D03A8DD097243ACD5620D8
:10263000E3EB152D54F6D4297926A9C5CE3B68C104
:10264000171D2BCCA000EAC8A550ADD6124D6CD2F8
:10265000CB6B2FDF7C76EEDBC1CBA1E376D660E7D8
:10266000AFF023EA18EDE2EE1DBDA5F0AAA064F4D8
:10267000738627F9C49BE6FD09FDB889BEE0798D14
:1026800067C63A80D0DBFB84D58BBC9A62967D9E70
:10269000BBB03E930CADFF97B110B0AF060D71AB60
:1026A000DF2B32A66836F3A26D66B4BCDA7B75B850
:1026B000035D36B5B440F7B1D8260008000000200D
:1026C00064000000A41E00083C27000864000020ED
:1026D0004C1D0000B41E00080000000000000000B7
:1026E0000000000000A24A040000000000000000FA
:1026F0000000000055AA07150C0BC1094D432056D8
:10270000312E322E3200000000F055AA07150C05BC
:10271000A90341434B00000000F055AA07150C0423
:102720000000000000000000F00000001507000895
:0C2730000000000000000000AE050020CA
:04000005080000ED02
:00000001FF
